:100000000C94A1000C94C22A0C94ED2A0C94182B89
:100010000C94CB000C94CB000C94CB000C94CB0034
:100020000C94CB000C94CB000C94CB000C94CB0024
:100030000C94CB000C94CB000C94CB000C94CB0014
:100040000C94CB000C94CB000C94E1280C94CB00C6
:100050000C94E1260C9417270C94CB000C94CB0045
:100060000C94CB000C94CB000C94CB000C94CB00E4
:100070000C94CB000C94CB000C94CB000C94CB00D4
:100080000C94CB000C94CB000C94CB0056213A215D
:1000900059213D2140214321462149214D21512112
:1000A000F429F729EA29EE290E2A0E2AFB29FF292D
:1000B000052A092A8B2B902B952B9F2BCD2BCD2BF3
:1000C000A92BB12BB92BC32B000000010200090A98
:1000D000000000000403080700000000000000000A
:1000E0000000000000000000010204081020408011
:1000F0000102040810204080010204081020408002
:1001000001020408102040800202020202020202E0
:1001100004040404040404040303030303030303A7
:100120000101010101010101000022002500280058
:100130002B0000002100240027002A00C505EC2424
:100140004B2711241FBECFEFD0E4DEBFCDBF11E09F
:10015000A0E0B1E0E0E1FCE500E00BBF02C00790E9
:100160000D92AE34B107D9F729E3AEE4B1E001C096
:100170001D92A933B207E1F710E0C1EAD0E004C054
:100180002197FE010E94912CCE39D107C9F70E9418
:1001900079270C94062E0C9400000F931F93CF9395
:1001A000DF931F92CDB7DEB78C0169830E94E82DE3
:1001B0006981681741F0C8010F90DF91CF911F91BD
:1001C0000F910C94F02D0F90DF91CF911F910F9113
:1001D00008950C94E82DDC01ED91FC910190F081E3
:1001E000E02D099461E08CE00C944B2A60E08CE0F7
:1001F0000C944B2A61E08DE00C944B2A60E08DE07A
:100200000C944B2A1F93CF93DF93EC0111E0892BC1
:1002100011F010E022C0C1E0D0E01FC061E08CE02E
:100220000E944B2A60E08DE00E944B2A64E670E059
:1002300080E090E00E945C2960E08CE00E944B2A04
:1002400061E08DE00E944B2A64E670E080E090E07F
:100250000E945C29111101C021971C161D06F4F2A1
:1002600060E08CE00E944B2A60E08DE0DF91CF914E
:100270001F910C944B2A1F93CF93DF93EC0111E055
:10028000892B11F010E002C0C1E0D0E061E08DE008
:100290000E944B2A60E08DE01C161D06B4F40E94FB
:1002A0004B2A64E670E080E090E00E945C2961E007
:1002B0008DE00E944B2A64E670E080E090E00E94AE
:1002C0005C291111E7CF2197E5CFDF91CF911F91E5
:1002D0000C944B2A1F93CF93DF93EC0111E0892BF1
:1002E00011F010E018C0C1E0D0E015C00E944B2A08
:1002F00064E670E080E090E00E945C2961E08CE0C0
:100300000E944B2A64E670E080E090E00E945C2945
:10031000111101C0219760E08CE01C161D0634F31A
:10032000DF91CF911F910C944B2A80914E019091B7
:100330004F01A0915001B09151010196A11DB11D35
:1003400080934E0190934F01A0935001B0935101BF
:1003500040910401509105016091060170910701DF
:10036000481759076A077B0720F510924E01109233
:100370004F011092500110925101609153018091F0
:100380000901861710F081E005C080910801681707
:1003900018F08FEF8093520180915201680F6093A3
:1003A000530170E08CE00E94642B60E08DE00C94BF
:1003B0004B2A089580914E0190914F01A0915001D8
:1003C000B09151010196A11DB11D80934E019093F2
:1003D0004F01A0935001B0935101409104015091FD
:1003E00005016091060170910701481759076A07D6
:1003F0007B0720F510924E0110924F011092500190
:10040000109251016091530180910901861710F0FB
:1004100081E005C080910801681718F08FEF809384
:10042000520180915201680F6093530170E08DE09A
:100430000E94642B60E08CE00C944B2A089560ECE1
:1004400070E08FE898E30E94EB0066E070E08FE8D0
:1004500098E30E94EB006091623870E08FE898E3C7
:100460000E94EB0060EC70E08FE898E30C94EB00E6
:1004700060EC70E08FE898E30E94EB0067E070E0CA
:100480008FE898E30E94EB006091190170E08FE81B
:1004900098E30E94EB0060EC70E08FE898E30C9426
:1004A000EB0060EC70E08FE898E30E94EB006FE0F7
:1004B00070E08FE898E30E94EB0061E070E08FE865
:1004C00098E30E94EB0060EC70E08FE898E30C94F6
:1004D000EB0060EC70E08FE898E30E94EB006EE0C8
:1004E00070E08FE898E30E94EB00809160388823E9
:1004F00019F061E070E002C060E070E08FE898E31E
:100500000E94EB0060EC70E08FE898E30C94EB0045
:1005100060EC70E08FE898E30E94EB0068E070E028
:100520008FE898E30E94EB0066E470E08FE898E3C0
:100530000E94EB0060EC70E08FE898E30C94EB0015
:1005400060EC70E08FE898E30E94EB0060E570E0FB
:100550008FE898E30E94EB0061E070E08FE898E399
:100560000E94EB0066E070E08FE898E30E94EB00E9
:1005700060EC70E08FE898E30C94EB0080916238B7
:10058000882341F060916B3870916C388DE698E368
:100590000C942423089580916238882341F060915F
:1005A0001C0170911D018DE698E30C9400240895C0
:1005B000809162388823E1F080915F38843A51F469
:1005C00060911A0170911B0140E050E08DE698E3C4
:1005D0000E94CD2480915F38893A51F460911A01CC
:1005E00070911B0141E050E08DE698E30C94CD241E
:1005F000089580916238882361F08DE698E30E9427
:100600002921609367387093683880936938909394
:100610006A38089580916238882371F04091673874
:10062000509168386091693870916A388DE698E326
:100630000E9460230C94F902089580916238882307
:1006400061F08DE698E30E94F9206093633870931F
:100650006438809365389093663808958091623845
:10066000882371F040916338509164386091653807
:10067000709166388DE698E30E9461220C941D0308
:10068000089580916238882321F08DE698E30C94D8
:100690005E2180E0089583ED9FE00E94E90091E0F3
:1006A000833709F090E0892F0895C8E3DFE06FEF0A
:1006B000CE010E94CD002196C11580E1D807B9F77F
:1006C0000E94FA000E94F600FBCF83ED9FE00E949B
:1006D000E90091E0833709F090E0892F089588E3DD
:1006E0009FE00E94E90091E0833009F090E0892FBB
:1006F000089589E39FE00E94E900982F80935F3876
:1007000081E0943A21F0993A11F080E0089508953B
:100710008AE39FE00E94E90080935E389FEF980F84
:1007200081E09E3F08F080E00895BF92CF92DF9273
:10073000EF92FF920F931F93CF93DF938BE090E0A4
:100740000E94B4277C018C01C0E0D0E0CE01885C1F
:10075000904F0E94E900F80181938F012196CB30E0
:10076000D105A1F76BE070E0C7010E94C51FB82E4C
:10077000C92E082F192FC0E0D0E0DD24D394CE017C
:100780008D5B904F0E94E900F80191918F018913D0
:10079000D12C2196C031D10591F78B2D9C2D0E9433
:1007A0004928C7010E9449288D2DDF91CF911F91C3
:1007B0000F91FF90EF90DF90CF90BF9008958FED55
:1007C0009FE00E94E90091E0833709F090E0892FD3
:1007D0000895CF92DF92EF92FF92CF930E94DF03B2
:1007E000882309F463C084ED9FE00E94E90090E053
:1007F00090936C3880936B3885ED9FE00E94E90000
:1008000090E090931D0180931C0186ED9FE00E9473
:10081000E90090E090931B0180931A018BED9FE01B
:100820000E94E900C82F8CED9FE00E94E900C82ECD
:10083000D12CE12CF12C7601DD24CC24FC2A8DED89
:100840009FE00E94E900C82F8EED9FE00E94E90022
:10085000C82ADC2AC0926338D0926438E0926538A6
:10086000F092663887ED9FE00E94E900C82F88ED7E
:100870009FE00E94E900C82ED12CE12CF12C7601DA
:10088000DD24CC24FC2A89ED9FE00E94E900C82FDA
:100890008AED9FE00E94E900C82ADC2AC0926738EE
:1008A000D0926838E0926938F0926A38CF91FF9020
:1008B000EF90DF90CF90089580916138882309F4FC
:1008C0008AC080916238882309F485C060916B38B2
:1008D00084ED9FE00E94CD0060911C0185ED9FE0BA
:1008E0000E94CD0060911A0186ED9FE00E94CD002C
:1008F0008091673890916838A0916938B0916A38D2
:100900006B2F77278827992787ED9FE00E94CD00DE
:100910008091673890916838A0916938B0916A38B1
:10092000BD018827992788ED9FE00E94CD00809126
:10093000673890916838A0916938B0916A38692F0A
:100940007A2F8B2F992789ED9FE00E94CD0060912F
:1009500067388AED9FE00E94CD00809163389091C6
:100960006438A0916538B09166386B2F7727882757
:1009700099278BED9FE00E94CD0080916338909184
:100980006438A0916538B0916638BD0188279927F1
:100990008CED9FE00E94CD00809163389091643887
:1009A000A0916538B0916638692F7A2F8B2F9927DF
:1009B0008DED9FE00E94CD00609163388EED9FE049
:1009C0000E94CD0063E78FED9FE00E94CD008AE09A
:1009D00090E00C946A018AE090E00C943B0160E0A6
:1009E0008FED9FE00C94CD0082E390E00E94020125
:1009F0000E9455038DE698E30E945D2210926238B2
:100A000008958091633890916438A0916538B091D1
:100A10006638892B8A2B8B2BE1F080916738909177
:100A20006838A0916938B0916A38892B8A2B8B2B52
:100A300081F080911A0190911B018F3F910549F03F
:100A400080916B3890916C38892B19F010921901B4
:100A5000089581E080931901089581E040916B0130
:100A600050916C012091690130916A01421753073E
:100A700009F480E0089580916B0190916C010196DA
:100A800069E170E00E943C2CAC0181E02091690199
:100A900030916A014217530709F080E00895CF931F
:100AA0008DE698E30E94A620C82F0E942B29609310
:100AB0005D0170935E0180935F0190936001C0FFC0
:100AC00004C081E08093680102C010926801109216
:100AD00067011092660120916801809161019091F7
:100AE0006201211108C00097E1F001979093620123
:100AF0008093610118C02091130130911401821775
:100B0000930748F40196909362018093610181E01C
:100B1000809365010AC081E0809365018093640140
:100B200004C01092640110926501809164018823D1
:100B300019F0CF910C94F200CF910C94F6000F9322
:100B40001F930E942B2900915D0110915E0120915D
:100B50005F0130916001DC01CB01801B910BA20B86
:100B6000B30B00910F0110911001209111013091F0
:100B7000120180179107A207B30720F01F910F9170
:100B80000C944F051F910F91089580910901809356
:100B900053010895803C41F46BED70E08FE898E3D9
:100BA0000E94EB008CED09C08B3D39F46BED70E0D9
:100BB0008FE898E30E94EB008DED682F8FE898E3B3
:100BC0000C942F2660EC70E08FE898E30E94EB0015
:100BD00061E270E08FE898E30E94EB00809174017D
:100BE0000E94CA05809173010E94CA05809172011A
:100BF0000E94CA05809171010E94CA0560EC70E0F4
:100C00008FE898E30C94EB0060EC70E08FE898E3D9
:100C10000E94EB0062E270E08FE898E30E94EB0034
:100C2000809170010E94CA0580916F010E94CA05DF
:100C300080916E010E94CA0580916D010E94CA05D3
:100C400060EC70E08FE898E30C94EB0060EC70E0EF
:100C50008FE898E30E94EB0062E070E08FE898E391
:100C60000E94EB0080916A380E94CA058091693821
:100C70000E94CA05809168380E94CA058091673831
:100C80000E94CA0560EC70E08FE898E30C94EB00DA
:100C900060EC70E08FE898E30E94EB0061E070E0A8
:100CA0008FE898E30E94EB00809166380E94CA05A5
:100CB000809165380E94CA05809164380E94CA05F7
:100CC000809163380E94CA0560EC70E08FE898E379
:100CD0000C94EB00CF93DF93C8E3DFE0CE010E94DA
:100CE000E9000E94CA052196C11580E1D807B1F735
:100CF000DF91CF91089560EC70E08FE898E30E9457
:100D0000EB0061E570E08FE898E30E94EB000E9441
:100D10006A0660EC70E08FE898E30C94EB00CF93E8
:100D2000C82F60EC70E08FE898E30E94EB0060E968
:100D300070E08FE898E30E94EB006C2F8FE898E357
:100D40000E942F2660EC70E08FE898E3CF910C941E
:100D5000EB001F93CF93DF931F92CDB7DEB7182F11
:100D600069830E944B036981811102C0183C38F0ED
:100D700083E00F90DF91CF911F910C948F06812F0C
:100D800090E0885C904F0F90DF91CF911F910C9471
:100D9000CD000E94010580916238811144C080918C
:100DA000190181113CC0809161388823C1F14091C3
:100DB00063385091643860916538709166388DE67B
:100DC00098E30E94B922892B41F481E00E948F06AA
:100DD00080E090E00E940201089581E080936238F3
:100DE0000E94D8020E940A030E94BE020E94CB0207
:100DF0000E941D038DE698E30E94232465E27AE0B9
:100E00008DE698E30E94F12160E070E08DE698E3C2
:100E10000E94752483E090E00E946A01089583E0B7
:100E200090E00E943B0108950E946503882361F0D1
:100E30000E946F03882341F00E947903882321F0E8
:100E40000E948803811103C01092613808950E94A6
:100E50009503882371F081E0809361380E94DF035D
:100E6000882339F00E94E90382E1809318010C94F1
:100E7000C906089580E00E94432B0E94882726E03F
:100E800040E052EC61E070E08FE898E30E94762643
:100E900061E08CE00E940F2A61E08DE00E940F2A41
:100EA00084EF91E0E7E6F6E3DF019C011D9221501B
:100EB0003040E1F7E3E7F4E3DF019C011D922150AC
:100EC0003040E1F710926F34109270341092713408
:100ED0001092723484ED90E3E7EAF1E0DF019C01C7
:100EE0001D9221503040E1F782E3E5E7F1E0DF01B8
:100EF0001D928A95E9F722E030E043E050E064E09B
:100F000070E08DE698E30E9444200C941407CF9380
:100F1000DF93EC0120916B0130916C01C9010196C6
:100F200069E170E00E943C2C4091690150916A0196
:100F30008417950721F1F901EE0FFF1FEB58FE4FC3
:100F4000D183C08344EF51E0249FF001259FF00D31
:100F5000349FF00D1124E955FE4FA3E7B4E39D0142
:100F6000235734432C173D0718F42D912193F7CFC5
:100F700090936C0180936B01DF91CF91089584E091
:100F8000DF91CF910C948F06CF93C0911601CC5D69
:100F900060EC70E08FE898E30E94EB0063E270E0A1
:100FA0008FE898E30E94EB006C2F8FE898E30E9493
:100FB0002F2660EC70E08FE898E3CF910C94EB0063
:100FC00060EC70E08FE898E30E94EB0064E070E072
:100FD0008FE898E30E94EB0060916B388FE898E30C
:100FE0000E942F2660EC70E08FE898E30C94EB00F1
:100FF00060EC70E08FE898E30E94EB0065E070E041
:101000008FE898E30E94EB0060911C018FE898E361
:101010000E942F2660EC70E08FE898E30C94EB00C0
:1010200060EC70E08FE898E30E94EB0063E070E012
:101030008FE898E30E94EB0060911A018FE898E333
:101040000E942F2660EC70E08FE898E30C94EB0090
:10105000CF93C82F60EC70E08FE898E30E94EB001C
:1010600060E470E08FE898E30E94EB006C2F8FE85B
:1010700098E30E942F2660EC70E08FE898E3CF9110
:101080000C94EB0090915A01992371F0803CD1F4BB
:1010900080910E0181110BC010925A0180915B0169
:1010A00090915C010C948707803C09F0ACC181E011
:1010B00080935A018EEF80930E0110925C01109282
:1010C0005B01089520915B0130915C01243F91E028
:1010D000390708F098C190910E012115310529F4C6
:1010E0009E3F19F480930E01089591111FC08B3D0E
:1010F00021F481E080935901089590915901992339
:1011000049F08C3D21F08D3D19F48BED01C080EC50
:1011100010925901A9014F5F5F4F50935C014093BA
:101120005B01F901ED58FB4C80830895913009F083
:101130004AC08B3D19F49093590118C09091590100
:10114000992349F08C3D21F08D3D19F48BED01C0C0
:1011500080EC10925901A9014F5F5F4F50935C01E1
:1011600040935B01F901E159FB4C808380915B0165
:1011700090915C01049709F046C120916F348091F1
:10118000703490E0A0E0B0E0DC0199278827B22B12
:1011900020917234822B20917134922B0097A105FB
:1011A000B10511F40C944806809363389093643829
:1011B000A0936538B093663880911801813191F71A
:1011C0000E942E03EFCF923009F04BC08B3D21F4EB
:1011D00081E08093590118C090915901992349F0F9
:1011E0008C3D21F08D3D19F48BED01C080EC109207
:1011F0005901A9014F5F5F4F50935C0140935B0120
:10120000F901E159FB4C808380915B0190915C0175
:10121000049709F0F8C020916F348091703490E009
:10122000A0E0B0E0DC0199278827B22B209172342E
:10123000822B20917134922B0097A105B10511F4F6
:101240000C9426068093673890936838A093693889
:10125000B0936A3880911801813191F70E940A0396
:10126000EFCF9330A9F48F3F11F40C941008823122
:1012700010F490E002C081E190E090931B01809314
:101280001A0180911801813181F70E94D802EDCFB7
:101290009430D1F48F3F11F40C94E007873038F08C
:1012A000282F30E08D3028F02CE030E002C027E01D
:1012B00030E030936C3820936B3880911801813185
:1012C00059F70E94BE02E8CF9530D1F48F3F11F458
:1012D0000C94F807853038F0282F30E0893028F05A
:1012E00028E030E002C025E030E030931D0120937B
:1012F0001C0180911801813159F70E94CB02E8CF7F
:10130000963071F48F3F21F0811104C00E94FA04DD
:101310000C941F02813009F076C00E94C906F8CFF4
:10132000913211F40C94E205923211F40C940406FB
:10133000933211F40C94C407973021F40E940105F4
:101340000C943802903319F490E00C946A019034B4
:1013500021F40E9441030C942808983029F4833723
:1013600009F051C00C9488029E3059F4813019F470
:101370008093603804C0811102C0109260380C94D0
:101380006902993521F4883FF1F50E94F404913502
:1013900011F40C947B06923551F58B3D21F481E0DC
:1013A0008093590118C090915901992349F08C3DBF
:1013B00021F08D3D19F48BED01C080EC10925901A4
:1013C000A9014F5F5F4F50935C0140935B01F901AE
:1013D000E159FB4C808380915B0190915C01029705
:1013E00091F46091703480916F340C94A90690351B
:1013F00011F40C94A002933511F40C945C04943510
:1014000011F40C94EF0408950F931F93CF93DF937F
:101410008C0101151105A1F0C0915B38D0915C38A9
:10142000CE01019690935C3880935B388DE698E30B
:101430000E94DE20C959D94C888301501109E9CF97
:10144000DF91CF911F910F9108950F931F93CF9329
:10145000DF938C018DE698E30E94A92080935D388C
:101460008091603881112CC08DE698E30E94DE20C7
:101470009C01015011098091150120FF0CC03327F8
:1014800094E0359527959A95E1F78F3F09F494C03C
:10149000821392C077C08F3F39F010925C3810925F
:1014A0005B388FEF809315018DE698E30E94AC20A6
:1014B0009093170180931601C8010E94040A91C0FD
:1014C00010925C3810925B388DE698E30E94AC2055
:1014D0009093170180931601C8010E94040A60ECE2
:1014E00070E08FE898E30E94EB0063E270E08FE821
:1014F00098E30E94EB006091160164528FE898E334
:101500000E942F2660EC70E08FE898E30E94EB00C9
:1015100060E070E08FE898E30E94EB00C7E6D6E356
:1015200020915B3830915C38CE0187569643821704
:10153000930778F060EC70E08FE898E30E94EB008E
:1015400010925C3810925B38DF91CF911F910F9110
:1015500008956991603C41F46BED70E08FE898E389
:101560000E94EB006CED09C06B3D39F46BED70E04F
:101570008FE898E30E94EB006DED8FE898E30E94FE
:101580002F26CECFC0911601D09117018DE698E39A
:101590000E94AC208C0F9D1F97FD01969C013595F4
:1015A00027953093170120931601C8010E94040A61
:1015B0008FEF8093150115C010925C3810925B3844
:1015C000209315018DE698E30E94AC2090931701BB
:1015D00080931601C801DF91CF911F910F910C9458
:1015E000040A60EC70E08FE898E30E94EB0063E28D
:1015F00070E08FE898E30E94EB006091160164525E
:101600008FE898E30E942F2660EC70E08FE898E363
:101610000E94EB0060E070E08FE898E30E94EB002E
:10162000C7E6D6E320915B3830915C38CE0187560F
:1016300096438217930708F07DCF6991603C41F48F
:101640006BED70E08FE898E30E94EB006CED09C051
:101650006B3D39F46BED70E08FE898E30E94EB008E
:101660006DED8FE898E30E942F26DCCFCF92DF92BA
:10167000EF92FF920F931F93CF93DF93EC01809132
:101680006238882309F47AC080916038811158C08B
:101690000E94FA0060E071E080E090E00E949027F4
:1016A000162F107FCF3FD10508F0116060E070E089
:1016B0008DE698E30E945424612F8DE698E30E9402
:1016C000FE1F9BE7C92E92E3D92EEE24E394F12C62
:1016D000C6018B5792438C179D07F0F4F601619178
:1016E0006F018DE698E30E94FE1FFFEFEF1AFF0ADD
:1016F0008FEFE816F10461F78DE698E30E9461210F
:1017000060E070E08DE698E30E945424612F8DE63E
:1017100098E30E94FE1FD9CF8DE698E30E946121D5
:101720000E94FE0060E070E08DE698E3DF91CF91CB
:101730001F910F91FF90EF90DF90CF900C94752444
:101740000E94FA00CF3FD10519F010F0CFEFD0E0A2
:1017500060E070E08DE698E30E9454240BE712E30A
:10176000C8018B5792438C179D07B0F6F801619121
:101770008F018DE698E30E94FE1FF2CF82E00E9467
:101780008F0685E090E0DF91CF911F910F91FF9040
:10179000EF90DF90CF900C940201CF93DF932091D4
:1017A000690130916A0184EF91E0289FF001299F3F
:1017B000F00D389FF00D1124A901440F551FDA01D7
:1017C000AB58BE4FCD91DC91ABE7B2E3E955FE4F8C
:1017D000BF01CF01861B970B8C179D0720F48081DA
:1017E0008D931192F6CFFA01EB58FE4F11821082C1
:1017F000C901019669E170E00E943C2C90936A0156
:1018000080936901CE010E94360B0E943B05811135
:1018100004C0DF91CF910C945102DF91CF910895D4
:101820000F931F9380916238882359F00E949F057F
:101830000E942D05882381F08091580181110CC0F0
:101840004AC080916138882319F00E94950104C034
:101850000E94DA010E94FA048FE898E30E949F2513
:10186000892BA1F081E0809358018FE898E30E94D2
:10187000B9250E9442080E942B296093540170935D
:10188000550180935601909357014CC080915801A7
:10189000882309F447C00E942B290091540110911C
:1018A00055012091560130915701DC01CB01801B7D
:1018B000910BA20BB30B00910A0110910B01209127
:1018C0000C0130910D0180179107A207B30750F169
:1018D0001092580127C080916301811102C00E94BB
:1018E0004F0580916501811119C0809164018111BA
:1018F00015C080916301882331F062E370E080E0DD
:1019000090E00E945C290E944F0580916501811141
:10191000A3CF109263010E94CD0B9ECF81E08093F4
:1019200063019ACF1F910F9108952F923F924F928A
:101930005F926F927F928F929F92AF92BF92CF925F
:10194000DF92EF92FF920F931F93CF93DF93CDB768
:10195000DEB7C058D1090FB6F894DEBF0FBECDBFB9
:10196000C158DF4F99838883CF57D04067965FAFC8
:101970004EAF6797DC0118964D905D906D907C900E
:101980001B9765964CAE5DAE6EAE7FAE65971C96AE
:101990004D905D906D907C901F9749825A826B822A
:1019A0007C8250964D905D906D907C9053974D82C7
:1019B0005E826F82788654964D905D906D907C909B
:1019C00057974D865E866F86788A605C7F4FA85AEF
:1019D000BF4F6996BFAFAEAF6997FC01E45AFF4FA6
:1019E0006B96FFAFEEAF6B979C01205A3F4F6D9601
:1019F0003FAF2EAF6D978C599F4F6F969FAF8EAFB5
:101A00006F97C158DF4FA881B981CF57D040A859EF
:101A1000BF4FA196BFAFAEAFA197C158DF4FE881CE
:101A2000F981CF57D040E459FF4FA396FFAFEEAFF7
:101A3000A397C158DF4F28813981CF57D040205913
:101A40003F4FA5963FAF2EAFA597C158DF4F888176
:101A50009981CF57D0408C589F4FA7969FAF8EAF9C
:101A6000A797C158DF4FA881B981CF57D040A85858
:101A7000BF4FA996BFAFAEAFA997C158DF4F28801F
:101A80003980CF57D040BCE72B0E311CC158DF4FF7
:101A9000E881F981CF57D040E058FF4FAB96FFAFB8
:101AA000EEAFAB97C158DF4F28813981CF57D04077
:101AB0002C573F4FAD963FAF2EAFAD97C158DF4F7C
:101AC00088819981CF57D04088579F4FAF969FAF5D
:101AD0008EAFAF97C158DF4FA881B981CF57D040A3
:101AE000A457BF4FE196BFAFAEAFE197C158DF4FEC
:101AF000E881F981CF57D040E057FF4FE396FFAF21
:101B0000EEAFE397C158DF4F28813981CF57D040DE
:101B10002C563F4FE5963FAF2EAFE597E6966FAF59
:101B2000E697E7967FAFE797FB01FF9780813196B5
:101B30008080912CA12CB12C540199248824982ABE
:101B400032978081882A3396808124013501782A52
:101B5000498A5A8A6B8A7C8A6996AEADBFAD69970D
:101B60004D925D926D927C92139765968CAD9DAD72
:101B7000AEADBFAD659788589B45A549B8428D84E9
:101B80009E84AF84B8884D805E806F807884842482
:101B90009524A624B724C980DA80EB80FC808C20B1
:101BA0009D20AE20BF202D853E854F8558898226F9
:101BB0009326A426B526880E991EAA1EBB1E8989C7
:101BC0009A89AB89BC89880E991EAA1EBB1ED501B5
:101BD000C40127E0880F991FAA1FBB1F2A95D1F7C0
:101BE00039E1B694A794979487943A95D1F7882AC7
:101BF000992AAA2ABB2A8C0C9D1CAE1CBF1C3296AB
:101C000080813196008110E020E030E098011127BA
:101C10000027182B32978081082B3396808128016A
:101C20003901782A4D8A5E8A6F8A788E6B96AEADBE
:101C3000BFAD6B974D925D926D927C9213974D84E0
:101C40005E846F847888BAEA4B1AB8E45B0AB8E31A
:101C50006B0AB7E17B0A8D899E89AF89B88D840DA7
:101C6000951DA61DB71D4D805E806F8078844C2425
:101C70005D246E247F24482059206A207B20CD805B
:101C8000DE80EF80F8844C245D246E247F24480E8F
:101C9000591E6A1E7B1ED301C2015CE0880F991F8A
:101CA000AA1FBB1F5A95D1F714E1769467945794F5
:101CB00047941A95D1F7482A592A6A2A7B2A480C50
:101CC000591C6A1C7B1C329680813196C080D12CB5
:101CD000E12CF12C7601DD24CC24D82A32978081A6
:101CE000C82A33968081A7019601582B298F3A8FF5
:101CF0004B8F5C8F6D96AEADBFAD6D972D933D93C1
:101D00004D935C931397CD80DE80EF80F884B5E22D
:101D1000CB1ABFE8DB0ABFEDEB0ABBEDFB0ADA0129
:101D2000C9018C0D9D1DAE1DBF1DC980DA80EB80E1
:101D3000FC80C824D924EA24FB24C420D520E62032
:101D4000F72029813A814B815C81C226D326E42683
:101D5000F526C80ED91EEA1EFB1ED701C6012FE0CC
:101D6000B695A795979587952A95D1F731E1CC0C33
:101D7000DD1CEE1CFF1C3A95D1F7C82AD92AEA2AA5
:101D8000FB2AC40CD51CE61CF71C32962081319628
:101D9000808190E0A0E0B0E0DC0199278827922BB9
:101DA00032972081822B3396E0819C01AD015E2B1E
:101DB0002D8F3E8F4F8F58A36F96AEADBFAD6F97EF
:101DC0002D933D934D935C93139709811A812B8139
:101DD0003C810251114322443E438D8D9E8DAF8D37
:101DE000B8A1800F911FA21FB31F93018201082584
:101DF00019252A253B250C211D212E213F210825AF
:101E000019252A253B25080F191F2A1F3B1FD90119
:101E1000C8015AE0B695A795979587955A95D1F739
:101E2000E6E1000F111F221F331FEA95D1F7082B9F
:101E3000192B2A2B3B2B0C0D1D1D2E1D3F1DFB01AD
:101E4000BF97408131965081852F90E0A0E0B0E0AF
:101E5000DC0199278827942B32974081842B339675
:101E60004081B42B89A39AA3ABA3BCA3A196EEADEA
:101E7000FFADA19780839183A283B3838155904F57
:101E8000A348BA40880E991EAA1EBB1ED701C601E0
:101E900084259525A625B72580239123A223B32346
:101EA00084259525A625B725880E991EAA1EBB1E3A
:101EB000D501C401E7E0880F991FAA1FBB1FEA954F
:101EC000D1F7F9E1B694A79497948794FA95D1F74E
:101ED000882A992AAA2ABB2A800E911EA21EB31E06
:101EE000FB01BB97408131965081852F90E0A0E0A7
:101EF000B0E0DC0199278827942B32974081842B0E
:101F000033964081B42B8DA39EA3AFA3B8A7A3960D
:101F1000EEADFFADA39780839183A283B383865DEB
:101F20009943A847B84B480E591E6A1E7B1ED9011B
:101F3000C8018C259D25AE25BF2588219921AA2180
:101F4000BB218C259D25AE25BF25480E591E6A1E36
:101F50007B1ED301C201ECE0880F991FAA1FBB1F93
:101F6000EA95D1F7F4E17694679457944794FA95FB
:101F7000D1F7482A592A6A2A7B2A480C591C6A1C1C
:101F80007B1CFB01B797408131965081852F90E0F3
:101F9000A0E0B0E0DC0199278827942B329740819C
:101FA000842B33964081B42B89A79AA7ABA7BCA7F3
:101FB000A596EEADFFADA59780839183A283B383F1
:101FC0008D5E994BAF4CB745C80ED91EEA1EFB1E5D
:101FD000D501C40180279127A227B3278421952109
:101FE000A621B72180279127A227B327C80ED91E83
:101FF000EA1EFB1ED701C601EFE0B695A79597959F
:102000008795EA95D1F7F1E1CC0CDD1CEE1CFF1CA5
:10201000FA95D1F7C82AD92AEA2AFB2AC40CD51C7A
:10202000E61CF71CFB01B397408131965081852F48
:1020300090E0A0E0B0E0DC0199278827942B32974C
:102040004081842B33964081B42B8DA79EA7AFA7E8
:10205000B8ABA796EEADFFADA79780839183A2831F
:10206000B3838F5F9A46A94BB240080F191F2A1FEE
:102070003B1FD301C20188259925AA25BB258C21A8
:102080009D21AE21BF2188259925AA25BB25080FB2
:10209000191F2A1F3B1FD901C801EAE0B695A79571
:1020A00097958795EA95D1F7F6E1000F111F221F4A
:1020B000331FFA95D1F7082B192B2A2B3B2B0C0D2C
:1020C0001D1D2E1D3F1DFB017F97408131965081C4
:1020D000852F90E0A0E0B0E0DC0199278827942BC1
:1020E00032974081842B33964081B42B89AB9AABD5
:1020F000ABABBCABA996EEADFFADA9978083918346
:10210000A283B38388529746AF47B649880E991E7B
:10211000AA1EBB1ED701C60184259525A625B72575
:1021200080239123A223B32384259525A625B725B3
:10213000880D991DAA1DBB1D4C015D01E7E0880CAF
:10214000991CAA1CBB1CEA95D1F7F9E1B695A79595
:1021500097958795FA95D1F788299929AA29BB29B6
:10216000800F911FA21FB31FFB017B974081319607
:102170005081852E912CA12CB12C540199248824B6
:10218000942A32974081842A33964081B42A8DAABA
:102190009EAAAFAAB8AEF10180829182A282B382D8
:1021A000F1E58F1AF8E09F0AFBEBAF0AF4E7BF0AEC
:1021B000480C591C6A1C7B1C480159018C249D2425
:1021C000AE24BF2488229922AA22BB228C249D24DB
:1021D000AE24BF24840C951CA61CB71C2401350119
:1021E000ECE0440C551C661C771CEA95D1F7F4E131
:1021F000B694A79497948794FA95D1F78428952854
:10220000A628B728880E991EAA1EBB1EFB01779729
:10221000408131965081452E512C612C712C320118
:1022200055244424542A32974081442A33964081CD
:10223000742A49AE5AAE6BAE7CAEAB96EEADFFAD36
:10224000AB974082518262827382FFE44F1AF4EAB4
:102250005F0A61087108C40CD51CE61CF71C2C0130
:102260003D014026512662267326482059206A20C7
:102270007B204026512662267326C40CD51CE61C02
:10228000F71C26013701EFE0769467945794479442
:10229000EA95D1F7F1E1CC0CDD1CEE1CFF1CFA95A0
:1022A000D1F7C428D528E628F728C80CD91CEA1C81
:1022B000FB1CFB017397408131965081452E512CB8
:1022C000612C712C320155244424542A32974081C8
:1022D000442A33964081742A21964CAE5DAE6EAE90
:1022E0007FAE2197AD96EEADFFADAD9740825182A6
:1022F00062827382F2E44F1AF8E25F0AF3EA6F0A2D
:10230000F6E77F0A040D151D261D371D2401350132
:10231000482659266A267B264C205D206E207F2089
:10232000482659266A267B26040D151D261D371DB5
:1023300028013901EAE07694679457944794EA9526
:10234000D1F7F6E1000F111F221F331FFA95D1F7C5
:1023500004291529262937290C0D1D1D2E1D3F1D69
:10236000FB013F97408131965081452E512C612CC5
:10237000712C320155244424542A32974081442A36
:1023800033964081742A25964CAE5DAE6EAE7FAE1C
:102390002597AF96EEADFFADAF9740825182628236
:1023A0007382FEED4F1AFEEE5F0AFFE66F0AF4E954
:1023B0007F0A840D951DA61DB71D260137014824EF
:1023C00059246A247B244022512262227322482409
:1023D00059246A247B24840D951DA61DB71D2C014C
:1023E0003D01E7E0440C551C661C771CEA95D1F7CB
:1023F000F9E1B695A79597958795FA95D1F7842930
:102400009529A629B729800F911FA21FB31FFB0191
:102410003B97408131965081452E512C612C712C77
:10242000320155244424542A32974081442A339659
:102430004081742A29964CAE5DAE6EAE7FAE299770
:10244000E196EEADFFADE1974082518262827382E8
:10245000FDE64F1AFEE85F0AF7E66F0AF2E07F0A30
:10246000840C951CA61CB71C280139014C245D2442
:102470006E247F24482259226A227B224C245D2428
:102480006E247F24840C951CA61CB71C24013501E6
:10249000ECE0440C551C661C771CEA95D1F7F4E17E
:1024A000B694A79497948794FA95D1F784289528A1
:1024B000A628B728880E991EAA1EBB1EFB013797B7
:1024C000408131965081452E512C612C712C320166
:1024D00055244424542A32974081442A339640811B
:1024E000742A2D964CAE5DAE6EAE7FAE2D97E39600
:1024F000EEADFFADE3974082518262827382F2E7D4
:102500004F1AFCEB5F0AF6E86F0AF9E57F0AC40C84
:10251000D51CE61CF71C2C013D01402651266226E5
:102520007326482059206A207B20402651266226A7
:102530007326C40CD51CE61CF71C26013701EFE0FE
:102540007694679457944794EA95D1F7F1E1CC0CCF
:10255000DD1CEE1CFF1CFA95D1F7C428D528E6280F
:10256000F728C80CD91CEA1CFB1CFB0133974081DF
:1025700031965081452E512C612C712C32015524FD
:102580004424542A32974081442A33964081742A45
:1025900061964CAE5DAE6EAE7FAE6197E596EEADE8
:1025A000FFADE5974082518262827382FFED4F1A40
:1025B000F7EF5F0AFBE46F0AF6EB7F0A040D151DC7
:1025C000261D371D24013501482659266A267B26FB
:1025D0004C205D206E207F20482659266A267B26C7
:1025E000040D151D261D371D28013901EAE07694DA
:1025F000679457944794EA95D1F7F6E1000F111FBD
:10260000221F331FFA95D1F70429152926293729C6
:102610000C0D1D1D2E1D3F1D4D885E886F88788C0A
:102620004EE9441A4AED540A41EE640A49E0740A3C
:10263000840D951DA61DB71D280139014C245D246C
:102640006E247F24482059206A207B204C245D245E
:102650006E247F24840D951DA61DB71D2C013D0100
:1026600045E0440C551C661C771C4A95D1F75BE18C
:10267000B695A795979587955A95D1F78429952969
:10268000A629B729800F911FA21FB31F49A45AA4DE
:102690006BA47CA450EC451A5CE4550A5FEB650A18
:1026A0005FE3750A840C951CA61CB71C2C013D0128
:1026B00040265126622673264C205D206E207F2006
:1026C0004026512662267326840C951CA61CB71C36
:1026D00024013501E9E0440C551C661C771CEA9581
:1026E000D1F7F7E1B694A79497948794FA95D1F728
:1026F00084289528A628B728880E991EAA1EBB1ED6
:1027000021964CAC5DAC6EAC7FAC2197EFEA4E1AD3
:10271000E5EA5E0AE1EA6E0AE9ED7E0AC40CD51C20
:10272000E61CF71C24013501482659266A267B261B
:102730004022512262227322482659266A267B268D
:10274000C40CD51CE61CF71C260137014EE0440CD6
:10275000551C661C771C4A95D1F752E1F694E79414
:10276000D794C7945A95D1F7C428D528E628F728D6
:10277000C80CD91CEA1CFB1C49885A886B887C88C9
:10278000F6E54F1AF8E35F0AF9E46F0AF6E17F0A0B
:10279000040D151D261D371D260137014824592417
:1027A0006A247B24482259226A227B224824592405
:1027B0006A247B24040D151D261D371D28013901AF
:1027C000ECE07694679457944794EA95D1F7F4E156
:1027D000000F111F221F331FFA95D1F70429152965
:1027E000262937290C0D1D1D2E1D3F1D4DA05EA055
:1027F0006FA078A443EA441A4FEE540A40ED640AED
:1028000049E2740A840D951DA61DB71D28013901E2
:102810004C245D246E247F24482059206A207B208C
:102820004C245D246E247F24840D951DA61DB71DA8
:102830002C013D0145E0440C551C661C771C4A9553
:10284000D1F75BE1B695A795979587955A95D1F7FE
:1028500084299529A629B729800F911FA21FB31F8C
:1028600049AC5AAC6BAC7CAC5DEA451A5BEE550AE0
:102870005BEB650A5DEF750A840C951CA61CB71C02
:102880002C013D0140265126622673264C205D20F6
:102890006E207F204026512662267326840C951CCC
:1028A000A61CB71C24013501E9E0440C551C661C2C
:1028B000771CEA95D1F7F7E1B694A794979487949B
:1028C000FA95D1F784289528A628B728880E991E4E
:1028D000AA1EBB1E61964CAC5DAC6EAC7FAC619722
:1028E000EFE74E1AE9E15E0AEEE56E0AE7E27E0ADC
:1028F000C40CD51CE61CF71C2401350148265926BA
:102900006A267B26402251226222732248265926BB
:102910006A267B26C40CD51CE61CF71C2601370151
:102920004EE0440C551C661C771C4A95D1F752E1C9
:10293000F694E794D794C7945A95D1F7C428D5282C
:10294000E628F728C80CD91CEA1CFB1C49A05AA091
:102950006BA07CA0F8E34F1AF4E05F0AFCE26F0A78
:10296000F8E17F0A040D151D261D371D26013701CC
:10297000482459246A247B24482259226A227B2233
:10298000482459246A247B24040D151D261D371D57
:1029900028013901ECE07694679457944794EA95BE
:1029A000D1F7F4E1000F111F221F331FFA95D1F761
:1029B00004291529262937290C0D1D1D2E1D3F1D03
:1029C0004DA85EA86FA878AC4AE1441A42E3540AC5
:1029D0004EE1640A4EED740A840D951DA61DB71DC7
:1029E000280139014C245D246E247F24482059207D
:1029F0006A207B204C245D246E247F24840D951D49
:102A0000A61DB71D2C013D0145E0440C551C661C5C
:102A1000771C4A95D1F75BE1B695A7959795879571
:102A20005A95D1F784299529A629B729800F911F96
:102A3000A21FB31F2D964CAC5DAC6EAC7FAC2D9736
:102A40005AE2451A58EF550A58EC650A5CE3750AD4
:102A5000840C951CA61CB71C2C013D014026512658
:102A6000622673264C205D206E207F204026512652
:102A700062267326840C951CA61CB71C2401350104
:102A8000E9E0440C551C661C771CEA95D1F7F7E188
:102A9000B694A79497948794FA95D1F784289528AB
:102AA000A628B728880E991EAA1EBB1E4D8C5E8CC8
:102AB0006F8C78A0E9E74E1AE2EF5E0AEAE26E0A4E
:102AC000EBE07E0AC40CD51CE61CF71C2401350182
:102AD000482659266A267B264022512262227322EA
:102AE000482659266A267B26C40CD51CE61CF71CF2
:102AF000260137014EE0440C551C661C771C4A9594
:102B0000D1F752E1F694E794D794C7945A95D1F748
:102B1000C428D528E628F728C80CD91CEA1CFB1CB9
:102B200049A85AA86BA87CA8F3E14F1AFBEE5F0AEC
:102B3000F5EA6F0AFAEB7F0A040D151D261D371DF5
:102B400026013701482459246A247B24482259222B
:102B50006A227B22482459246A247B24040D151DF3
:102B6000261D371D28013901ECE0769467945794AF
:102B70004794EA95D1F7F4E1000F111F221F331F8C
:102B8000FA95D1F704291529262937292801390171
:102B90004C0C5D1C6E1C7F1CEB964CAE5DAE6EAE9D
:102BA0007FAEEB9729964CAC5DAC6EAC7FAC2997B1
:102BB0002BEF421A26E1520A2CE1620A26E5720A3C
:102BC000840D951DA61DB71DEB964CAC5DAC6EAC8F
:102BD0007FACEB974C245D246E247F244820592041
:102BE0006A207B204C245D246E247F24840D951D57
:102BF000A61DB71D2C013D0115E0440C551C661C9B
:102C0000771C1A95D1F70BE1B695A79597958795FF
:102C10000A95D1F784299529A629B729EB964CACBA
:102C20005DAC6EAC7FACEB97840D951DA61DB71DFA
:102C3000498C5A8C6B8C7C8C28E0421A2CE5520A09
:102C400020E1620A23E0720A840C951CA61CB71CC2
:102C5000EB964CAC5DAC6EAC7FACEB97482659263E
:102C60006A267B264C205D206E207F20EB962CADC3
:102C70003DAD4EAD5FADEB974226532664267526DB
:102C8000840C951CA61CB71C2401350129E0440CBA
:102C9000551C661C771C2A95D1F737E1B694A7948A
:102CA000979487943A95D1F784289528A628B72831
:102CB000880E991EAA1EBB1E4DA45EA46FA478A800
:102CC00037E2431A3DEF530A30E9630A38E9730AE1
:102CD000C40CD51CE61CF71C2401350148265926D6
:102CE0006A267B26EB962CAD3DAD4EAD5FADEB97E6
:102CF0004222532264227522482659266A267B26C0
:102D0000C40CD51CE61CF71C260137014EE0440C10
:102D1000551C661C771C4A95D1F752E1F694E7944E
:102D2000D794C7945A95D1F7C428D528E628F72810
:102D3000C80CD91CEA1CFB1C260137014824592465
:102D40006A247B24EF964CAE5DAE6EAE7FAEEF97FD
:102D500025964CAC5DAC6EAC7FAC259726E7421A4D
:102D600023EB520A25ED620A22E7720AEB962CAD9C
:102D70003DAD4EAD5FADEB97420E531E641E751E0A
:102D8000EF962CAD3DAD4EAD5FADEF9728233923C7
:102D90004A235B23282539254A255B25420E531EED
:102DA000641E751EA3019201ECE056954795379578
:102DB0002795EA95D1F729873A874B875C87930156
:102DC0008201F4E1000F111F221F331FFA95D1F782
:102DD00049845A846B847C8404291529262937293F
:102DE000280139014C0C5D1C6E1C7F1CEB964CAE0F
:102DF0005DAE6EAE7FAEEB974DA05EA06FA078A4E7
:102E00002EEB421A26EC520A25E0620A7108840D64
:102E1000951DA61DB71DEF964CAC5DAC6EAC7FAC9E
:102E2000EF97EB962CAD3DAD4EAD5FADEB974226E7
:102E3000532664267526840D951DA61DB71D2C01ED
:102E40003D0114E0440C551C661C771C1A95D1F703
:102E50000CE1B695A795979587950A95D1F78429A2
:102E60009529A629B729820F931FA41FB51F49A82A
:102E70005AA86BA87CA83FE7431A39E0530A3EE8FA
:102E8000630A38E7730A840C951CA61CB71CEB96E2
:102E90004CAC5DAC6EAC7FACEB974C245D246E24E7
:102EA0007F24482659266A267B26840C951CA61C5E
:102EB000B71C240135012BE0440C551C661C771C03
:102EC0002A95D1F735E1B694A794979487943A95CB
:102ED000D1F784289528A628B728880E991EAA1EFF
:102EE000BB1E21964CAC5DAC6EAC7FAC21974EED19
:102EF000441A4EE9540A42E6640A42E9740AC40CD0
:102F0000D51CE61CF71CEB964CAC5DAC6EAC7FACF4
:102F1000EB97482659266A267B26482459246A249A
:102F20007B24C40CD51CE61CF71CF60167017F014D
:102F3000C80CD91CEA1CFB1C2D964CAC5DAC6EACCD
:102F40007FAC2D97F4EF4F1AF7EC5F0AFAE16F0AA6
:102F5000F2E07F0AEB960CAD1DAD2EAD3FADEB97C9
:102F6000040D151D261D371D24013501482659263F
:102F70006A267B264C245D246E247F24040D151DB7
:102F8000261D371D2801390149E07694679457942E
:102F900047944A95D1F757E1000F111F221F331FA5
:102FA0005A95D1F704291529262937290C0D1D1DFD
:102FB0002E1D3F1D4D885E886F88788C4CEB441A1F
:102FC00045E1540A41E4640A4BE5740A840D951DF9
:102FD000A61DB71D26013701482459246A247B24E5
:102FE0004026512662267326840D951DA61DB71D09
:102FF0002C013D01E4E0440C551C661C771CEA954D
:10300000D1F7FCE1B695A79597958795FA95D1F7F5
:1030100084299529A629B729800F911FA21FB31FC4
:1030200049A05AA06BA07CA057E5451A50E3550A69
:1030300051E2650A54EB750A840C951CA61CB71C5A
:10304000280139014C245D246E247F24482659260A
:103050006A267B26840C951CA61CB71C240135010E
:103060004BE0440C551C661C771C4A95D1F755E182
:10307000B694A794979487945A95D1F78428952865
:10308000A628B728880E991EAA1EBB1E4DA45EA4B2
:103090006FA478A8E0EA4E1AE4EB5E0AE4E46E0A54
:1030A000E9E07E0AC40CD51CE61CF71C2C013D018E
:1030B0004026512662267326482459246A247B24FC
:1030C000C40CD51CE61CF71C260167017201C80C54
:1030D000D91CEA1CFB1C49AC5AAC6BAC7CAC40E97B
:1030E000441A43E4540A40E4640A41E4740A040DB7
:1030F000151D261D371D24013501482659266A262F
:103100007B264C245D246E247F24040D151D261D72
:10311000371D28013901E9E0769467945794479464
:10312000EA95D1F7F7E1000F111F221F331FFA951F
:10313000D1F704291529262937290C0D1D1D2E1D0F
:103140003F1D29964CAC5DAC6EAC7FAC29975AE321
:10315000451A51E8550A54E6650A57ED750A840D7B
:10316000951DA61DB71D26013701482459246A2440
:103170007B244026512662267326480E591E6A1E5D
:103180007B1ED301C20144E0880F991FAA1FBB1FF9
:103190004A95D1F75CE176946794579447945A9591
:1031A000D1F7482A592A6A2A7B2A400E511E621EEC
:1031B000731E89899A89AB89BC898650984DAE4522
:1031C000B541880E991EAA1EBB1ED901C8018C25C7
:1031D0009D25AE25BF2584259525A625B725880DD7
:1031E000991DAA1DBB1D4C015D01EBE0880C991CCB
:1031F000AA1CBB1CEA95D1F7F5E1B695A795979562
:103200008795FA95D1F788299929AA29BB29840D90
:10321000951DA61DB71D8D8C9E8CAF8CB8A0EBE7BD
:103220008E1AEFEC9E0AE0E1AE0AEBE2BE0AC80C91
:10323000D91CEA1CFB1C5301420180269126A226C0
:10324000B32688269926AA26BB26C80CD91CEA1CB8
:10325000FB1C460167017401C80ED91EEA1EFB1E45
:1032600089A49AA4ABA4BCA44BEF841A42EE940A9E
:1032700047E7A40A4BEFB40A080D191D2A1D3B1D90
:103280004C015D0184249524A624B7248C249D241C
:10329000AE24BF24080D191D2A1D3B1D48015901EC
:1032A00049E0B694A794979487944A95D1F757E14B
:1032B000000F111F221F331F5A95D1F70829192912
:1032C0002A293B290C0D1D1D2E1D3F1D8DA89EA8D2
:1032D000AFA8B8AC57EC851A5FE2950A5BE2A50A85
:1032E00056E2B50A480C591C6A1C7B1C4601570162
:1032F00088269926AA26BB2680269126A226B326B2
:10330000480C591C6A1C7B1C53014201E4E0880CE8
:10331000991CAA1CBB1CEA95D1F7FCE17694679432
:1033200057944794FA95D1F7482859286A287B285A
:10333000400E511E621E731E25968CAC9DACAEAC29
:10334000BFAC2597EBE18E1AE6E69E0AE4E2AE0AF0
:10335000E9E1BE0A880D991DAA1DBB1D480159014E
:103360008C249D24AE24BF2484249524A624B72431
:10337000880D991DAA1DBB1D4C015D014BE0880CF9
:10338000991CAA1CBB1C4A95D1F755E1B695A79587
:10339000979587955A95D1F788299929AA29BB2904
:1033A000840D951DA61DB71D61968CAC9DACAEAC71
:1033B000BFAC6197F8E08F1AF3E89F0AFDE5AF0A0A
:1033C000F0EEBF0AC80CD91CEA1CFB1C53014201D9
:1033D00080269126A226B32688269926AA26BB26D1
:1033E000C80CD91CEA1CFB1C460167017401C80EFD
:1033F000D91EEA1EFB1E898C9A8CAB8CBC8C4BE9C7
:10340000841A49EA940A43E5A40A4BE3B40A080D76
:10341000191D2A1D3B1D4C015D0184249524A62401
:10342000B7248C249D24AE24BF24080D191D2A1D09
:103430003B1D48015901E9E0B694A79497948794FD
:10344000EA95D1F7F7E1000F111F221F331FFA95FC
:10345000D1F7082919292A293B290C0D1D1D2E1DDC
:103460003F1D89889A88AB88BC885CEB851A5DED26
:10347000950A56EDA50A5BE0B50A480C591C6A1C72
:103480007B1C4C015D0180949094A094B094802AA0
:10349000912AA22AB32A8C249D24AE24BF24480C4E
:1034A000591C6A1C7B1C5301420146E0880C991C84
:1034B000AA1CBB1C4A95D1F75AE17694679457949D
:1034C00047945A95D1F7482859286A287B28400EF6
:1034D000511E621E731E8DA49EA4AFA4B8A8E9E677
:1034E0008E1A9108E5EDAE0AECEBBE0A880D991D27
:1034F000AA1DBB1D4601570180949094A094B094DE
:1035000084289528A628B72880269126A226B326A7
:10351000880D991DAA1DBB1D4C015D01EAE0880CB8
:10352000991CAA1CBB1CEA95D1F7F6E1B695A795A4
:1035300097958795FA95D1F788299929AA29BB29C2
:10354000840D951DA61DB71D2D968CAC9DACAEAC03
:10355000BFAC2D97F9E58F1AFCED9F0AFBE6AF0A89
:10356000F4E5BF0AC80CD91CEA1CFB1C4801590130
:1035700080949094A094B094882A992AAA2ABB2A6D
:1035800084249524A624B724C80CD91CEA1CFB1C4F
:10359000460157014FE0880C991CAA1CBB1C4A9598
:1035A000D1F751E1F694E794D794C7945A95D1F79F
:1035B000C828D928EA28FB28C80ED91EEA1EFB1EF7
:1035C0008DA09EA0AFA0B8A447EC841A4FE5940A42
:1035D0004CE6A40A43E0B40A080D191D2A1D3B1D40
:1035E0005301420180949094A094B0948C289D281B
:1035F000AE28BF2888269926AA26BB26080D191DA5
:103600002A1D3B1D48015901EBE0B694A7949794FD
:103610008794EA95D1F7F5E1000F111F221F331FA0
:10362000FA95D1F7082919292A293B290C0D1D1DC6
:103630002E1D3F1D25968CAC9DACAEACBFAC259726
:103640005DE3851A56EA950A54EAA50A5AE9B50ACD
:10365000480C591C6A1C7B1C4C015D0180949094A1
:10366000A094B094802A912AA22AB32A8C249D2463
:10367000AE24BF24480C591C6A1C7B1C5301420118
:1036800046E0880C991CAA1CBB1C4A95D1F75AE14C
:1036900076946794579447945A95D1F748285928B7
:1036A0006A287B28400E511E621E731E8D8C9E8CD4
:1036B000AF8CB8A0EEE68E1AE3E39E0AE3EFAE0A03
:1036C000E0E7BE0A880D991DAA1DBB1D46015701E2
:1036D00080949094A094B09484289528A628B72824
:1036E00080269126A226B326880D991DAA1DBB1DF2
:1036F0004C015D01EAE0880C991CAA1CBB1CEA95F0
:10370000D1F7F6E1B695A79597958795FA95D1F7F4
:1037100088299929AA29BB29840D951DA61DB71DA5
:1037200089AC9AACABACBCACF3E88F1AFBE09F0A57
:10373000F0E1AF0AB108C80CD91CEA1CFB1C480117
:10374000590180949094A094B094882A992AAA2A26
:10375000BB2A84249524A624B724C80CD91CEA1CAF
:10376000FB1C460157014FE0880C991CAA1CBB1C8E
:103770004A95D1F751E1F694E794D794C7945A95B6
:10378000D1F7C828D928EA28FB28C80ED91EEA1E76
:10379000FB1E8D889E88AF88B88C4FE2841A42EA5F
:1037A000940A4BE7A40A4AE7B40A080D191D2A1D1A
:1037B0003B1D5301420180949094A094B0948C28B6
:1037C0009D28AE28BF2888269926AA26BB26080D44
:1037D000191D2A1D3B1D48015901EBE0B694A79421
:1037E00097948794EA95D1F7F5E1000F111F221FF6
:1037F000331FFA95D1F7082919292A293B290C0DDD
:103800001D1D2E1D3F1D89A89AA8ABA8BCA851EB71
:10381000851A51E8950A57E5A50A50E9B50A480CFA
:10382000591C6A1C7B1C4C015D0180949094A094EF
:10383000B094802A912AA22AB32A8C249D24AE24F3
:10384000BF24840C951CA61CB71C2401350146E03E
:10385000440C551C661C771C4A95D1F75AE1B69466
:10386000A794979487945A95D1F784289528A628E9
:10387000B728800E911EA21EB31E61964CAC5DACA3
:103880006EAC7FAC6197E0E24E1AE9E15E0AE3EDCF
:103890006E0AE1E07E0A840D951DA61DB71D260166
:1038A00037014094509460947094482859286A28AD
:1038B0007B284026512662267326840D951DA61D61
:1038C000B71D2C013D01EAE0440C551C661C771C19
:1038D000EA95D1F7F6E1B695A79597958795FA956C
:1038E000D1F784299529A629B729880D991DAA1DE4
:1038F000BB1D49A45AA46BA47CA4FCEE4F1AFCEB9C
:103900005F0AFEEF6F0AFCE57F0AC40CD51CE61CBB
:10391000F71C280139014094509460947094482A0F
:10392000592A6A2A7B2A482459246A247B24C40CF5
:10393000D51CE61CF71C260137014FE0440C551C32
:10394000661C771C4A95D1F751E1F694E794D79419
:10395000C7945A95D1F7C428D528E628F728C80E69
:10396000D91EEA1EFB1E29964CAC5DAC6EAC7FAC3A
:1039700029974FE5441A4EEE540A47EF640A41EB8B
:10398000740A400E511E621E731E9501840100953B
:103990001095209530950C291D292E293F2908279F
:1039A00019272A273B27040D151D261D371D280121
:1039B0003901EBE07694679457944794EA95D1F7F0
:1039C000F5E1000F111F221F331FFA95D1F70429CB
:1039D0001529262937290C0D1D1D2E1D3F1D49A017
:1039E0005AA06BA07CA05EE7451A51E8550A5CEA34
:1039F000650A58E0750A840C951CA61CB71C2C019E
:103A00003D014094509460947094402A512A622A57
:103A1000732A4C245D246E247F24840C951CA61CE0
:103A2000B71C2401350146E0440C551C661C771C6C
:103A30004A95D1F75AE1B694A794979487945A95EA
:103A4000D1F784289528A628B728800E911EA21E9B
:103A5000B31E21964CAC5DAC6EAC7FAC2197EBEC09
:103A60004E1AEDE05E0AE5EC6E0AE2E47E0A840D91
:103A7000951DA61DB71D26013701409450946094F2
:103A80007094482859286A287B28402651266226A7
:103A90007326840D951DA61DB71D2C013D01EAE07E
:103AA000440C551C661C771CEA95D1F7F6E1B695D7
:103AB000A79597958795FA95D1F784299529A629F1
:103AC000B729880D991DAA1DBB1D498C5A8C6B8C7A
:103AD0007C8CF5E44F1AFDE25F0AF8E26F0AF5ED1F
:103AE0007F0AC40CD51CE61CF71C28013901409440
:103AF000509460947094482A592A6A2A7B2A482450
:103B000059246A247B24C40CD51CE61CF71C26010E
:103B100037014FE0440C551C661C771C4A95D1F7C1
:103B200051E1F694E794D794C7945A95D1F7C428F5
:103B3000D528E628F728C80ED91EEA1EFB1E4DA878
:103B40005EA86FA878AC4FE6441A4CE2540A49E7E5
:103B5000640A44E1740A040D151D261D371D240155
:103B6000350140945094609470944C285D286E28E0
:103B70007F28482659266A267B26040D151D261DFA
:103B8000371D28013901EBE07694679457944794E8
:103B9000EA95D1F7F5E1000F111F221F331FFA95A7
:103BA000D1F7042915292629372965964CAC5DAC37
:103BB0006EAC7FAC6597480C591C6A1C7B1C6596E3
:103BC0004CAE5DAE6EAE7FAE65970C0D1D1D2E1D0D
:103BD0003F1D69807A808B809C80600E711E821EE2
:103BE000931E69827A828B829C828D809E80AF80B8
:103BF000B8848C0C9D1CAE1CBF1C8D829E82AF8233
:103C0000B886AD84BE84CF84D888A80EB91ECA1EDB
:103C1000DB1EAD86BE86CF86D88A67962EAD3FADB9
:103C200067972054310967963FAF2EAF6797605C66
:103C30007F4F232B11F00C948E0D65968CAD9DADAE
:103C4000AEADBFAD6597C158DF4FE881F981CF5761
:103C5000D04080879187A287B38749805A806B8044
:103C60007C8044865586668677864D805E806F8030
:103C70007884408A518A628A738AA48AB58AC68AFD
:103C8000D78AE6968FADE697E7969FADE797C0583F
:103C9000DF4F0FB6F894DEBF0FBECDBFDF91CF91DF
:103CA0001F910F91FF90EF90DF90CF90BF90AF905A
:103CB0009F908F907F906F905F904F903F902F904C
:103CC0000895CF93DF93FC0181E093E2A5E4B7E68A
:103CD00080879187A287B38789E89BEAADECBFEE26
:103CE00084879587A687B7878EEF9CEDAAEBB8E906
:103CF000808B918BA28BB38B86E794E5A2E3B0E136
:103D0000848B958BA68BB78B1082118212821382C3
:103D10001482158216821782DF01A85ABF4F80E4F1
:103D2000ED01982F19929A95E9F77896DF011D9287
:103D30008A95E9F7DF91CF9108958F929F92AF9284
:103D4000BF92CF92DF92EF92FF920F931F93CF9388
:103D5000DF93EC016B017A01088119812A813B8193
:103D6000CA01A0E0B0E0AC01BD01400F511F621FCD
:103D7000731F7F71488359836A837B834017510780
:103D80006207730760F44C815D816E817F814F5FB4
:103D90005F4F6F4F7F4F4C835D836E837F830F73C5
:103DA000112722273327011511052105310549F176
:103DB00040E4842E912CA12CB12C801A910AA20AE5
:103DC000B30A085E1F4F88159905AA05BB0530F494
:103DD000A701B601CE01800F911F25C0A401B60135
:103DE000CE01800F911F0E94D82DC80CD91CE81855
:103DF000F90840E450E0BE01685E7F4FCE010E94AA
:103E0000950C80E4E816F10450F0A701407CB6015F
:103E1000CE010E94950C6C018FE3E822FF24A701DC
:103E2000B601CE014896DF91CF911F910F91FF907F
:103E3000EF90DF90CF90BF90AF909F908F900C94B9
:103E4000D82DCF92DF92EF92FF920F931F93CF93D3
:103E5000DF938C01EB01C880D980EA80FB802FE3DF
:103E6000C222DD24EE24FF24D701C6010196A11D44
:103E7000B11DFB01EC0DFD1D20E8208F4FE350E04C
:103E800060E070E04C195D096E097F09FE017896CB
:103E90007F014830510561057105A0F4489660E046
:103EA00070E08C0F9D1F0E94E12D40E450E0B701AF
:103EB000CE010E94950C40E450E060E070E080E0AC
:103EC00090E0DC0148505109489660E070E08C0FAA
:103ED0009D1F0E94E12D88819981AA81BB8123E0E9
:103EE000880F991FAA1FBB1F2A95D1F78883998332
:103EF000AA83BB83FE01E05BFF4F808331969083F2
:103F00003196A0833196B0833C812D819E818F8133
:103F10003196308331962083319690833196808319
:103F200040E450E0B701CE010E94950C8885F8016D
:103F30008083898581838A8582838B8583838C8531
:103F400084838D8585838E8586838F858783888905
:103F50008087898981878A8982878B8983878C89F1
:103F600084878D8985878E8986878F89878788E969
:103F7000FE0111928A95E9F7DF91CF911F910F9180
:103F8000FF90EF90DF90CF900895CF92DF92EF9265
:103F9000FF920F931F93CF93DF93CDB7DEB7C8592E
:103FA000D1090FB6F894DEBF0FBECDBF7C016B0107
:103FB00080E190E00E94B4278C01CE0101960E941E
:103FC000611EA601B701CE0101960E949D1EBE0191
:103FD0006F5F7F4FC8010E94211FC801C856DF4F85
:103FE0000FB6F894DEBF0FBECDBFDF91CF911F910A
:103FF0000F91FF90EF90DF90CF900895CF93DF93D4
:104000001F92CDB7DEB76983DC01ED91FC91028090
:10401000F381E02D41E050E0BE016F5F7F4F0995D5
:104020000F90DF91CF9108950895FC0113821282C1
:1040300088EE93E0A0E0B0E084839583A683B78305
:104040008FE291E09183808380E5848781E085879A
:104050008AE090E09787868789E090E0918B808B5B
:1040600082E090E0938B828B148A158A168A178AD5
:10407000118E108E138E128E158E148E40E050E02D
:10408000BA01CF010C94DB26FC0177876687518B40
:10409000408B338B228B0895EF92FF921F93CF9327
:1040A000DF931F92CDB7DEB77C01162F60E0FC01D5
:1040B000868549830E944B2AF70154853585809176
:1040C0008D384981882399F02FB7F89480918D38E5
:1040D000813059F48DB380938B389DB380918C38A7
:1040E000809589238DBB2FBF02C020938B385CBD88
:1040F0003DBD1EBD00000DB407FEFDCF8EB54EBD0B
:1041000000000DB407FEFDCF1EB580918D388823C9
:1041100061F08FB7F89420918D3890918B382130D1
:1041200019F49DBB8FBF01C09FBF61E0F701868579
:104130000E944B2A812F0F90DF91CF911F91FF900A
:10414000EF9008956F7740E00C944C2068E10C9458
:10415000A2206AE10C94A2200F931F93CF93DF93C8
:104160008C016AE10E94A220C82FD0E0F801648986
:104170007589868997890E94DD2B24ED30E843E418
:104180005EE40E94D62B87FD2797CE018D599109B9
:10419000DF91CF911F910F910895CF93DF93EC01A1
:1041A00063E10E94A220282F30E0888D998DA9011B
:1041B000481B590BCA01DF91CF910895CF93DF932C
:1041C000EC01E881F9810480F581E02D0995892BC6
:1041D00059F0888D998D0196998F888F60E0CE0176
:1041E0000E94A22090E002C08FEF9FEFDF91CF915D
:1041F00008950F931F93CF93DF93EC0166E00E9425
:10420000A220182F67E0CE010E94A220082F68E0AC
:10421000CE010E94A220402F50E060E070E0762F97
:10422000652F542F4427612B8A019B01082BC9015C
:10423000B80120E038E448EE51E00E94A52C03E1EB
:104240000E944A2DB901CA01DF91CF911F910F91B0
:1042500008956DE10E94A220E82FF0E084E0F5953A
:10426000E7958A95E1F7EA30F105F8F4EA5BFF4F4C
:104270000C94912C60EA78E21EC060E471E51BC0EA
:1042800062E17AE718C064EE72EA15C064E274EF86
:1042900012C068E478EE81E00FC060E970ED83E061
:1042A0000BC060E271EA87E007C0089568E77EE12D
:1042B00002C060EF7CE380E090E008956CE20C9433
:1042C000A220CF93DF93EC0143E861E80E944C20E9
:1042D00062E1CE010E94A22083FD03C00E947B2ADE
:1042E000F7CF48E062E9CE010E944C2081E090E0E7
:1042F000DF91CF9108958F929F92AF92BF92CF920C
:10430000DF92FF920F931F93CF93DF931F92CDB74E
:10431000DEB76C01B62E4A0162E279830E94A220C8
:10432000F82E90E09C01280D391D79812F3F310531
:1043300031F028F02FEF30E04901881A990A0B2D4F
:10434000172F5801A80CB91C0A151B0541F0F801DC
:1043500041918F0160E8C6010E944C20F5CF482DA5
:104360004F0D62EAC6010E944C20C4010F90DF91FC
:10437000CF911F910F91FF90DF90CF90BF90AF90A2
:104380009F908F900895EF92FF921F93CF93DF93AA
:104390001F92CDB7DEB77C01DC01ED91FC9104806A
:1043A000F581E02D0995892B99F06DE0C7010E94F8
:1043B000A220482F60E0C70149830E94A220182F45
:1043C00049816DE8C7010E944C20812F90E002C016
:1043D0008FEF9FEF0F90DF91CF911F91FF90EF90A4
:1043E0000895CF93DF93EC017D8F6C8F672BA9F13C
:1043F00060E08A890E940F2A40E060ECCE010E94B2
:104400004C208A899B898230910539F08A30910548
:1044100031F00B9731F08FEF05C082E003C080E0F0
:1044200001C081E00E943A258A899B8982309105EA
:1044300039F08A30910531F00B9731F08FEF05C0DC
:1044400082E003C080E001C081E043E050E069EC1D
:1044500074E2DF91CF910C947D2A8A899B89823006
:10446000910539F08A30910531F00B9731F08FEFDB
:1044700005C082E003C080E001C081E00E94AC2A58
:104480008A899B898230910539F08A30910531F013
:104490000B9731F08FEF05C082E003C080E001C0D0
:1044A00081E0DF91CF910C94592541E861E80C94AB
:1044B0004C2040E861E80C944C200E9459220C9456
:1044C00026258F929F92AF92BF92CF92DF92EF926A
:1044D000FF920F931F93CF93DF931F92CDB7DEB759
:1044E0004C01DB01CA01F401448B558B668B778B41
:1044F0006A017B01FF0CCC08DC2C76019A01AD012E
:104500006C2D7C2D8C2D9C2D03E10E942F2DA12C38
:10451000E8E4BE2EF8EECF2EDD24D394E12CF12C6E
:1045200000E010E00E94D22C69017A01A701662701
:10453000772766E8C40129830E944C2077276F2DD6
:104540005E2D4D2D67E8C4010E944C202981422F29
:1045500068E8C4010F90DF91CF911F910F91FF90F8
:10456000EF90DF90CF90BF90AF909F908F900C9482
:104570004C20CF92DF92EF92FF92CF93DF93EC012A
:104580006A017B0161E08E850E940F2A61E08E85C1
:104590000E944B2A888999898F3F2FEF9207B9F0A3
:1045A00061E00E940F2A60E088890E944B2A6AE03D
:1045B00070E080E090E00E945C2961E088890E94C0
:1045C0004B2A6AE070E080E090E00E945C290E9443
:1045D000F02462E4CE010E94A220823161F5CE0176
:1045E0000E945922B701A601CE010E94612240E03B
:1045F0006EE8CE010E944C2040E06FE8CE010E94A0
:104600004C206CE0CE010E94A220482F43606CE851
:10461000CE010E944C2044E066EACE010E944C206C
:1046200040E869E8CE010E944C20CE010E9455224C
:1046300081E090E002C080E090E0DF91CF91FF90B8
:10464000EF90DF90CF9008950F931F93CF93DF9358
:104650008C01EB016630710534F06D30710584F426
:104660006630710579F445EC61EBC8010E944C207D
:104670004CE067EBC8010E944C20C6E0D0E00CC0C3
:10468000CCE0D0E043EC61EBC8010E944C204AE052
:1046900067EBC8010E944C206EE1C8010E94A22075
:1046A00094E0CC0FDD1F9A95E1F78F704C2F482BCB
:1046B0006EE9C801DF91CF911F910F910C944C20AE
:1046C000CF92DF92EF92FF920F931F93CF93DF93DE
:1046D0008C01CB01BA010E94DD2B6B017C0120E033
:1046E00030EC43EF55E40E94D62B18160CF056C060
:1046F00020E030E842E256E4C701B6010E94D62B22
:1047000018160CF04EC020E030EC43E756E4C70129
:10471000B6010E94D62B18160CF046C020E030E8F7
:1047200042EA56E4C701B6010E94D62B18160CF0D7
:104730003EC020E034E244EF56E4C701B6010E94D7
:10474000D62B1816BCF520E034EE42E257E4C70140
:10475000B6010E94D62B181684F520E034E244E717
:1047600057E4C701B6010E94D62B18164CF520E07D
:1047700034E244EF57E4C701B6010E94D62B181665
:1047800014F520E034E244E758E4C701B6010E9482
:10479000D62B1816DCF4C9E0D0E01AC0C0E0D0E097
:1047A00017C0C1E0D0E014C0C2E0D0E011C0C3E047
:1047B000D0E00EC0C4E0D0E00BC0C5E0D0E008C03F
:1047C000C6E0D0E005C0C7E0D0E002C0C8E0D0E05D
:1047D0006DE1C8010E94A22094E0CC0FDD1F9A95E4
:1047E000E1F78F704C2F482B6DE9C801DF91CF9115
:1047F0001F910F91FF90EF90DF90CF900C944C2081
:104800000F931F93CF93DF938C01653071053CF0BC
:10481000EB01693071052CF0C8E0D0E002C0C5E0C2
:10482000D0E06DE1C8010E94A2202497CC0FDD1FCB
:10483000817F4C2F482B6DE9C801DF91CF911F91EB
:104840000F910C944C20CF93DF93EC016EE10E940A
:10485000A220482F44606EE9CE01DF91CF910C94E5
:104860004C20CF93DF93EC011B8E1A8E6DE10E94DA
:10487000A220482F4E7F6DE9CE01DF91CF910C949D
:104880004C20CF93DF93EC0181E090E09B8F8A8FE7
:104890006DE1CE010E94A220482F41606DE9CE015A
:1048A000DF91CF910C944C200F931F93CF93DF9304
:1048B000EC018B010E945522CE01012B19F00E94C0
:1048C000412402C00E94312440E06DE8CE010E94E4
:1048D0004C2040E062EACE010E944C2081E090E052
:1048E000DF91CF911F910F9108950F931F93CF9355
:1048F000DF93EC018B011616170644F40E94412445
:10490000402F62EACE010E944C2002C00E94312456
:1049100045E861E8CE01DF91CF911F910F910C9492
:104920004C201F93CF93DF93EC0162E10E94A22001
:10493000182F482F62E9CE010E944C2015FD25C09A
:10494000198E188E8A8D9B8D892B11F062E201C021
:1049500063E1CE010E94A220182F60E1CE010E94E7
:10496000A220482F6DE8CE010E944C20EC8DFD8DD9
:10497000309719F0812F90E0099540E06DE8CE0165
:10498000DF91CF911F910C944C20DF91CF911F911B
:1049900008958DE698E30C949124452B61F46F30D3
:1049A000710514F06EE070E077FF02C060E070E027
:1049B000462F40670EC06230710534F062317105D8
:1049C0002CF061E170E002C062E070E06250462FBE
:1049D000406869E80C944C208DE698E30C9415200F
:1049E000CF93CFB7F89480918E38811127C0ECE037
:1049F000F1E08491ECEEF0E09491E82FF0E0EE0F1E
:104A0000FF1FEE5CFE4FA591B491EC91E92321F4D8
:104A100061E084E00E944B2A61E084E00E940F2A5A
:104A20008CB580618CBD8CB580648CBD61E087E005
:104A30000E940F2A61E085E00E940F2A80918E3843
:104A40008F5F80938E38CFBFCF9108959FB7F89432
:104A500080918E38882319F0815080938E38809110
:104A60008E38811105C08CB58F7B8CBD10928D382E
:104A70009FBF08959FB7F894813029F058F0823095
:104A800021F484E008C082E006C082E080938D3883
:104A900080E001C081E020918C38822B80938C389B
:104AA00080918D38811103C081E080938D389FBF44
:104AB000089590918D389230B1F02FB7F8948330EB
:104AC00030F4E82FF0E0E55CFE4F808101C080E02B
:104AD000809590918C38892380938C38811102C005
:104AE00010928D382FBF0895CF92DF92EF92FF92F0
:104AF0000F931F93CF93DF936C017A018B01C0E07A
:104B0000D0E0CE15DF0589F0D8016D918D01D60179
:104B1000ED91FC910190F081E02DC6010995892B62
:104B200011F47E0102C02196ECCFC701DF91CF9135
:104B30001F910F91FF90EF90DF90CF900895FC01AF
:104B4000918D228D892F90E0805C9F4F821B91096F
:104B50008F7399270895FC01918D828D981731F0FC
:104B6000828DE80FF11D858D90E008958FEF9FEF06
:104B70000895FC01918D828D981761F0828DDF017F
:104B8000A80FB11D5D968C91928D9F5F9F73928F40
:104B900090E008958FEF9FEF089581E497E2892BCD
:104BA00041F080E090E0892B21F00E9441278111A3
:104BB0000DC080E090E0892B71F080E090E0892BBF
:104BC00051F00E940000811104C008950E9400006D
:104BD000F0CF0C9400000895FC01848DDF01A80F34
:104BE000B11DA35ABF4F2C91848D90E001968F7315
:104BF0009927848FA689B7892C93A089B1898C9134
:104C000080648C93938D848D981306C00288F389F9
:104C1000E02D80818F7D80830895CF93DF93EC0119
:104C2000888D8823C9F0EA89FB89808185FD05C0CC
:104C3000A889B9898C9186FD0FC00FB607FCF5CF06
:104C4000808185FFF2CFA889B9898C9185FFEDCF4E
:104C5000CE010E94EC25E7CFDF91CF910895EF922E
:104C6000FF920F931F93CF93DF93EC0181E0888F26
:104C70009B8D8C8D981305C0E889F989808185FD0D
:104C800024C0F62E0B8D10E00F5F1F4F0F731127FE
:104C9000E02E8C8DE8120CC00FB607FCFACFE88925
:104CA000F989808185FFF5CFCE010E94EC25F1CFF7
:104CB0008B8DFE01E80FF11DE35AFF4FF0820B8F41
:104CC000EA89FB898081806207C0EE89FF89608361
:104CD000E889F98980818064808381E090E0DF91B8
:104CE000CF911F910F91FF90EF900895CF92DF9297
:104CF000EF92FF921F93CF93DF93EC016A017B0148
:104D0000122FE889F98982E080834115514E6105AF
:104D10007105B1F060E079E08DE390E0A7019601C4
:104D20000E94502CDA01C9010197A109B109B69579
:104D3000A79597958795AC01411580E15807A8F094
:104D4000E889F989108260E874E88EE190E0A701B3
:104D500096010E94502CBA01A901415051096109E4
:104D600071097695679557954795EC85FD85508334
:104D7000EE85FF854083188EEC89FD891083EA89D2
:104D8000FB89808180618083EA89FB8980818860DA
:104D90008083EA89FB89808180688083EA89FB8936
:104DA00080818F7D8083DF91CF911F91FF90EF9065
:104DB000DF90CF900895FC01448355836683778309
:104DC00008951F920F920FB60F9211240BB60F92F7
:104DD0002F938F939F93EF93FF93E0919F38F091E0
:104DE000A0388081E091A538F091A63882FD12C0EC
:104DF00090818091A8388F5F8F732091A938821796
:104E000051F0E091A838F0E0E157F74C958F80938E
:104E1000A83801C08081FF91EF919F918F912F91D0
:104E20000F900BBE0F900FBE0F901F9018951F9202
:104E30000F920FB60F9211240BB60F922F933F9340
:104E40004F935F936F937F938F939F93AF93BF9392
:104E5000EF93FF938FE898E30E94EC25FF91EF9189
:104E6000BF91AF919F918F917F916F915F914F9182
:104E70003F912F910F900BBE0F900FBE0F901F9080
:104E800018958FE898E30E949F2521E0892B09F46B
:104E900020E0822F0895EFE8F8E31382128288EE73
:104EA00093E0A0E0B0E084839583A683B78382E497
:104EB00091E09183808385EC90E09587848784ECF2
:104EC00090E09787868780EC90E0918B808B81ECD7
:104ED00090E0938B828B82EC90E0958B848B86ECB8
:104EE00090E0978B868B118E128E138E148E089500
:104EF00008950E9498290E9478270E943A07CDECD5
:104F0000D5E20E94100C2097E1F30E94CD25F9CF45
:104F1000009729F0BC0180E090E00C94CF2D08951B
:104F2000CF93DF9300D000D0CDB7DEB76115710508
:104F30008105910579F09B01AC0169833A834B832C
:104F40005C830E94CB2D29813A814B815C810E9438
:104F5000722C03C060E070E0CB010F900F900F90B7
:104F60000F90DF91CF910895CF93DF938230910519
:104F700010F482E090E0E0913739F091383920E088
:104F800030E0C0E0D0E0309711F140815181481706
:104F90005907C0F04817590761F48281938120971F
:104FA00019F09B838A832BC09093383980933739CB
:104FB00026C02115310519F04217530718F49A013C
:104FC000BE01DF01EF010280F381E02DDCCF21156E
:104FD000310509F1281B390B2430310590F4129664
:104FE0008D919C9113976115710521F0FB019383BD
:104FF000828304C09093383980933739FD0132960B
:1050000044C0FD01E20FF31F8193919322503109B7
:105010002D933C933AC02091353930913639232B6A
:1050200041F42091200130912101309336392093B1
:10503000353920911E0130911F012115310541F4B0
:105040002DB73EB74091220150912301241B350B0F
:10505000E0913539F0913639E217F307A0F42E1BB1
:105060003F0B2817390778F0AC014E5F5F4F2417CC
:10507000350748F04E0F5F1F50933639409335394E
:105080008193919302C0E0E0F0E0CF01DF91CF91F6
:1050900008950F931F93CF93DF93009709F48CC06B
:1050A000FC013297138212820091373910913839FE
:1050B0000115110581F420813181820F931F209108
:1050C0003539309136392817390779F5F093363963
:1050D000E093353971C0D80140E050E0AE17BF070A
:1050E00050F412962D913C911397AD012115310585
:1050F00009F1D901F3CF9D01DA0133832283608165
:105100007181860F971F8217930769F4EC0128813C
:105110003981260F371F2E5F3F4F318320838A81CD
:105120009B8193838283452B29F4F0933839E09354
:10513000373942C01396FC93EE931297ED014991D3
:1051400059919E01240F351FE217F30771F48081F6
:105150009181840F951F029611969C938E93828164
:10516000938113969C938E931297E0E0F0E0D80120
:1051700012968D919C911397009719F0F8018C016C
:10518000F6CF8D919C9198012E5F3F4F820F931F18
:1051900020913539309136392817390769F430971D
:1051A00029F4109238391092373902C013821282D2
:1051B0001093363900933539DF91CF911F910F91BC
:1051C00008951F920F920FB60F9211242F933F93C1
:1051D0008F939F93AF93BF9380912D3990912E39E8
:1051E000A0912F39B091303930912C3923E0230F21
:1051F0002D3720F40196A11DB11D05C026E8230F0F
:105200000296A11DB11D20932C3980932D399093C6
:105210002E39A0932F39B093303980913139909144
:105220003239A0913339B09134390196A11DB11DA5
:105230008093313990933239A0933339B093343914
:10524000BF91AF919F918F913F912F910F900FBE82
:105250000F901F9018952FB7F89460912D39709189
:105260002E3980912F39909130392FBF08953FB753
:10527000F8948091313990913239A0913339B091BD
:10528000343926B5A89B05C02F3F19F00196A11D02
:10529000B11D3FBFBA2FA92F982F8827820F911DCC
:1052A000A11DB11DBC01CD0142E0660F771F881F13
:1052B000991F4A95D1F708958F929F92AF92BF920E
:1052C000CF92DF92EF92FF926B017C010E9437290F
:1052D0004B015C01C114D104E104F10401F10E940D
:1052E0007B2A0E943729DC01CB0188199909AA0978
:1052F000BB09883E9340A105B10560F321E0C21AC5
:10530000D108E108F10888EE880E83E0981EA11C00
:10531000B11CC114D104E104F10419F7DBCFFF90F3
:10532000EF90DF90CF90BF90AF909F908F900895B7
:10533000789484B5826084BD84B5816084BD85B570
:10534000826085BD85B5816085BDEEE6F0E0808137
:1053500081608083E1E8F0E0108280818260808358
:10536000808181608083E0E8F0E0808181608083DB
:10537000E1EBF0E0808184608083E0EBF0E080810D
:1053800081608083E1E9F0E08081826080838081B8
:1053900081608083E0E9F0E0808181608083EAE7DA
:1053A000F0E080818460808380818260808380815E
:1053B000816080838081806880831092C10008951D
:1053C00090E0FC013197EA30F10540F5E05BFF4FDA
:1053D0000C94912C809180008F7703C08091800085
:1053E0008F7D80938000089584B58F7702C084B547
:1053F0008F7D84BD08958091B0008F7703C0809128
:10540000B0008F7D8093B0000895809190008F77D9
:1054100003C0809190008F7D809390000895CF937A
:10542000DF9390E0FC01E851FF4F2491FC01E85F1D
:10543000FE4F8491882361F190E0880F991FFC0151
:10544000EE5CFE4FC591D491FC01E85DFE4FA59145
:10545000B491611109C09FB7F89488812095822387
:105460008883EC912E230BC0623061F49FB7F894CF
:105470003881822F809583238883EC912E2B2C9367
:105480009FBF06C08FB7F894E8812E2B28838FBF6B
:10549000DF91CF9108951F93CF93DF93282F30E0B2
:1054A000F901E853FF4F8491F901E851FF4FD4917E
:1054B000F901E85FFE4FC491CC23C9F0162F81118A
:1054C0000E94E029EC2FF0E0EE0FFF1FE85DFE4F99
:1054D000A591B4918FB7F894111105C09C91ED2F4F
:1054E000E095E92302C0EC91ED2BEC938FBFDF91A7
:1054F000CF911F91089508950895833060F5E82FA6
:10550000F0E0EE0FFF1FEC5DFE4F71836083813092
:1055100051F08230A1F0809169008C7F482B40933C
:105520006900E89A089580916900440F551F440F5F
:10553000551F837F482B40936900E99A0895809115
:10554000690094E0440F551F9A95E1F78F7C482B32
:1055500040936900EA9A0895833098F4813021F0ED
:10556000823021F0E89803C0E99801C0EA98E82F5A
:10557000F0E0EE0FFF1FEC5DFE4F8CE79AE29183A7
:10558000808308951F920F920FB60F9211240BB6CD
:105590000F922F933F934F935F936F937F938F93CC
:1055A0009F93AF93BF93EF93FF93E0912401F0910A
:1055B00025010995FF91EF91BF91AF919F918F9137
:1055C0007F916F915F914F913F912F910F900BBE03
:1055D0000F900FBE0F901F9018951F920F920FB64D
:1055E0000F9211240BB60F922F933F934F935F931B
:1055F0006F937F938F939F93AF93BF93EF93FF939B
:10560000E0912601F09127010995FF91EF91BF915B
:10561000AF919F918F917F916F915F914F913F914A
:105620002F910F900BBE0F900FBE0F901F901895EB
:105630001F920F920FB60F9211240BB60F922F9359
:105640003F934F935F936F937F938F939F93AF930A
:10565000BF93EF93FF93E0912801F0912901099501
:10566000FF91EF91BF91AF919F918F917F916F913A
:105670005F914F913F912F910F900BBE0F900FBEF6
:105680000F901F901895883028F0883110F08851BD
:1056900001C08FEF877020912A0190E4299F90012B
:1056A0001124822B80937C0080917A008064809307
:1056B0007A0080917A0086FDFCCF8091780020915D
:1056C000790090E0922B08951F93CF93DF93182FCA
:1056D000EB0161E00E940F2A209711F460E004C002
:1056E000CF3FD10539F461E0812FDF91CF911F9138
:1056F0000C944B2AE12FF0E0E853FF4FE4914E2F3A
:1057000050E0FA013197EA30F10508F046C0E65A58
:10571000FF4F0C94912C84B5806884BDC7BD42C0F6
:1057200084B5806284BDC8BD3DC080918000806822
:1057300080938000D0938900C093880033C080910B
:105740008000806280938000D0938B00C0938A0099
:1057500029C08091B00080688093B000C093B300EE
:1057600021C08091B00080628093B000C093B400EB
:1057700019C080919000806880939000D093990028
:10578000C09398000FC08091900080628093900039
:10579000D0939B00C0939A0005C0C038D1050CF08F
:1057A000A2CF9CCFDF91CF911F9108950E94182C1A
:1057B00008F481E00895E89409C097FB3EF49095C1
:1057C0008095709561957F4F8F4F9F4F9923A9F0DA
:1057D000F92F96E9BB279395F69587957795679569
:1057E000B795F111F8CFFAF4BB0F11F460FF1BC0AD
:1057F0006F5F7F4F8F4F9F4F16C0882311F096E940
:1058000011C0772321F09EE8872F762F05C06623ED
:1058100071F096E8862F70E060E02AF09A95660FA6
:10582000771F881FDAF7880F9695879597F908955F
:10583000990F0008550FAA0BE0E8FEEF16161706A1
:10584000E807F907C0F012161306E407F50798F009
:10585000621B730B840B950B39F40A2661F0232B22
:10586000242B252B21F408950A2609F4A140A6959E
:105870008FEF811D811D0895AA1BBB1B51E107C03D
:10588000AA1FBB1FA617B70710F0A61BB70B881FD0
:10589000991F5A95A9F780959095BC01CD0108955F
:1058A000A1E21A2EAA1BBB1BFD010DC0AA1FBB1F24
:1058B000EE1FFF1FA217B307E407F50720F0A21B96
:1058C000B30BE40BF50B661F771F881F991F1A9403
:1058D00069F760957095809590959B01AC01BD012D
:1058E000CF010895052E97FB1EF400940E94892C89
:1058F00057FD07D00E94502C07FC03D04EF40C94A7
:10590000892C50954095309521953F4F4F4F5F4FD3
:10591000089590958095709561957F4F8F4F9F4F1B
:105920000895EE0FFF1F0024001C0BBE0790F69198
:10593000E02D09940E94662DA59F900DB49F900DB7
:10594000A49F800D911D11240895E894DF93CF93B7
:10595000FC01DB010E94662D7F936F93E9019A01A0
:10596000AC01BF93AF933F932F93DF010E94662D4D
:1059700026F46C1B7D0B820B930B9E01EB01FC014B
:105980000E94752DAF91BF912F913F910E94752D6F
:10599000BE01CF01F9012F913F91CF91DF91089581
:1059A000689401C0E8948F929F92CF93DF930E94F6
:1059B000DE2CDF91CF919F908F90089588249924B9
:1059C000F401E401B0E49F93AA279A158B049C0488
:1059D000ED05FE05CF05D007A10798F4AD2FDC2F0C
:1059E000CF2FFE2FE92D982C892E982F872F762FD9
:1059F000652F542F432F322F2227B85031F7BF91F4
:105A000027C01B2EBF91BB27220F331F441F551FDA
:105A1000661F771F881F991F881C991CEE1FFF1F88
:105A2000CC1FDD1FAA1FBB1F8A149B04EC05FD05BC
:105A3000CE05DF05A007B10748F08A189B08EC09DE
:105A4000FD09CE09DF09A00BB10B21601A94E1F624
:105A50002EF49401AF01BE01CD01000C08950F9307
:105A6000083090F0982F872F762F652F542F432FD3
:105A7000322F22270850F4CF220F331F441F551F07
:105A8000661F771F881F991F0A95B2F70F91089517
:105A900097FB10F8169400080F93083098F0085000
:105AA000232F342F452F562F672F782F892F902D96
:105AB000F4CF059497958795779567955795479572
:105AC000379527950A95AAF70F910895A29FB001DF
:105AD000B39FC001A39F700D811D1124911DB29F22
:105AE000700D811D1124911D08950E94662D460F91
:105AF000571FC81FD91F08F4319608958F929F929F
:105B0000AF92BF92CF92DF92EF92FF92CF93DF934B
:105B1000EC01688179818A819B816115710581051C
:105B2000910521F464E279ED8BE597E02DE133EF07
:105B300041E050E00E94722C49015A019B01AC01E6
:105B4000A7EAB1E40E949A2C6B017C01ACEEB4EFA1
:105B5000A50194010E94012EDC01CB018C0D9D1D3D
:105B6000AE1DBF1DB7FF03C00197A109B0488883D0
:105B70009983AA83BB83BC01CD019F77DF91CF912D
:105B8000FF90EF90DF90CF90BF90AF909F908F905D
:105B900008950C947E2D80E091E00C947E2D60930E
:105BA0000001709301018093020190930301089515
:105BB000FB01DC0102C001900D9241505040D8F72A
:105BC0000895DC0101C06D9341505040E0F7089505
:105BD000F999FECF92BD81BDF89A992780B50895B5
:105BE000262FF999FECF1FBA92BD81BD20BD0FB6F9
:105BF000F894FA9AF99A0FBE01960895B7FF0C949B
:105C00009A2C0E949A2C821B930B0895F894FFCF34
:105C100001000000F82A0000160102000000FE0347
:105C20000000000F00FFDCFE1101FF000500000076
:105C3000393980007C2A7C2A7C2A0100000000FE81
:105C40001F7B21CD20DE20C321142001020400008F
:0E5C500000002F2674259F25B925AB250D26B3
:00000001FF
